:100000000C9455000C943A0B0C94670B0C94940BC5
:100010000C94C10B0C94EE0B0C941B0C0C94480C20
:100020000C94750C0C94ED060C949A050C94C00677
:100030000C9439060C9466060C946D050C949A0089
:100040000C947D000C947D000C94E2140C947D00C3
:100050000C947D140C947D000C947D000C947D0018
:100060000C9493060C94A1070C941A070C94470760
:100070000C9474070C940C060C94B6140C947D002C
:100080000C944F140C947D000C947D009D13000083
:100090000100080040000001000400000100080009
:1000A0002000400080000001000411241FBECFEF9B
:1000B000D0E1DEBFCDBF11E0A0E0B1E0E4E0F4E3C9
:1000C00000E00BBF02C007900D92A434B107D9F72E
:1000D00012E0A4E4B1E001C01D92A131B107E1F743
:1000E00010E0CEE8D0E004C02297FE010E94E4199F
:1000F000CC38D107C9F70C9460020C94000086B785
:10010000836086BF87B7826087BF87B78E7F87BFD0
:1001100080B7886080BF12BE80E281BF89E083BF64
:1001200080B7992787709070892BD1F786B7836045
:1001300086BF08951F920F920FB60F9211248F93CE
:100140009F93AF93BF938091C5019091C601A091F9
:10015000C701B091C8010196A11DB11D8093C501D1
:100160009093C601A093C701B093C8018091C901C3
:100170009091CA01A091CB01B091CC010196A11D33
:10018000B11D8093C9019093CA01A093CB01B09394
:10019000CC01BF91AF919F918F910F900FBE0F90A7
:1001A0001F9018956091C9017091CA018091CB018F
:1001B0009091CC0108959B01AC0112BE1092C50133
:1001C0001092C6011092C7011092C8018091C5011A
:1001D0009091C601A091C701B091C8018217930701
:1001E000A407B50799F70895019749F0880F991F5B
:1001F000880F991F0297F8940197F1F77894089562
:10020000E82FE695E695E695A82FBB27613081F4A7
:10021000FF27EE0FFF1FEA5EFE4F0190F081E02DF9
:10022000A770B070A050BF4F80819C91892B10C0E7
:10023000FF27EE0FFF1FEA5EFE4F0190F081E02DD9
:10024000A770B070A050BF4F9C919095808189237A
:1002500080830895A82F20E030E0E82FE695E6950A
:10026000E695FF27EE0FFF1FEC5DFE4F0190F0813A
:10027000E02DBB27A770B070A050BF4F80819C912C
:10028000892311F021E030E0C9010895E82FE695B7
:10029000E695E695A82FBB27613081F4FF27EE0F86
:1002A000FF1FE85FFE4F0190F081E02DA770B07056
:1002B000A050BF4F80819C91892B10C0FF27EE0F6B
:1002C000FF1FE85FFE4F0190F081E02DA770B07036
:1002D000A050BF4F9C919095808189238083089581
:1002E000E82FFF27613051F4EE0FFF1FEA5EFE4F4B
:1002F0000190F081E02D8FEF80830895EE0FFF1FB6
:10030000EA5EFE4F0190F081E02D10820895E82F03
:10031000FF27EE0FFF1FEC5DFE4F0190F081E02DF7
:10032000808199270895E82FFF27EE0FFF1FE85FD0
:10033000FE4F0190F081E02D6083089510926100DE
:100340001092620080E487B987EE86B9089597B16C
:10035000907E8770982B97B90895349BFECF0895AF
:10036000349A089584B195B1089597B1907E8770BD
:10037000982B97B9349A349BFECF349A20E030E022
:1003800040E008C0349BFECF84B195B1280F391FDF
:10039000349A4F5F4617B1F77727C9010E94911928
:1003A000CB010895CF93DF93E82FE695E695E69588
:1003B000FF27EE0FFF1FEC5DFE4F0190F081E02D57
:1003C000EF01A097992787709070A1E0B0E0082E08
:1003D00002C0AA0FBB1F0A94E2F720E030E06623B8
:1003E00011F021E030E002C0220F331F8A95E2F7BE
:1003F000332788A1682F77276A237B236217730727
:10040000C1F720E030E040E050E004C02F5F3F4FF4
:100410004F4F5F4F808199278A239B238617970729
:10042000A9F3CA01B90124E130E040E050E00E94A4
:10043000721927E130E040E050E00E94A519CA019E
:10044000B901DF91CF910895CF92DF92EF92FF92A1
:100450000F931F93CF93DF93E82EF62EC42ED22E48
:10046000C0E0D0E007E010E06D2D7727CC2039F414
:100470000C2E02C0759567950A94E2F706C0002E0F
:1004800002C0759567950A94E2F761708E2D0E94FF
:10049000460161E08F2D0E94460160E08F2D0E9491
:1004A0004601219601501040C830D105E9F6DF9190
:1004B000CF911F910F91FF90EF90DF90CF90089513
:1004C000CFEFD0E1DEBFCDBF0E947F00E0911C01E5
:1004D000F0911D018FEF8083E0911E01F0911F01CB
:1004E000808378940E94ED150E94D615FDCF982F39
:1004F00080913201813051F41092610010926200BB
:1005000080E487B987EE86B91092320163E0892FC3
:100510000E94B5010895853031F48FB580688FBD94
:100520008FB58F7B07C0843039F48FB580628FBD63
:100530008FB58F7E8FBD0895833031F48FB588607D
:100540008FBD8FB58B7FF6CF823049F480918B00C1
:10055000806880938B0080918B008F7B0AC08130F4
:1005600059F480918B00806280938B0080918B0086
:100570008F7E80938B000895882351F480918B00A7
:10058000886080938B0080918B008B7F80938B00A1
:1005900008958EB5887F83608EBD1DBC1CBC87B757
:1005A000846087BF089585B5887F826085BD14BC4F
:1005B00087B7806487BF1092D5011092D601109240
:1005C000D7011092D8011092D1011092D20110924D
:1005D000D3011092D4010895EAE8F0E08081887F89
:1005E000836080831092890010928800EDE7F0E02C
:1005F00080818460808308959EB5987F982B9EBDEE
:10060000089595B5987F982B95BD0895EAE8F0E098
:100610009081987F982B908308958E3040F4E82F36
:10062000FF27EE0FFF1FEB5BFE4F71836083089582
:10063000E3B7FF27E770F070EE0FFF1FE257FF4FA1
:10064000859194910895EEB5FF27E770F070EE0F55
:10065000FF1FE257FF4F859194910895E5B5FF275D
:10066000E770F070EE0FFF1FE257FF4F85919491F6
:100670000895E0918A00FF27E770F070EE0FFF1FEA
:10068000E257FF4F8591949108958E3040F4E82F02
:10069000FF27EE0FFF1FEB5BFE4F118210820895C4
:1006A000DF92EF92FF920F931F937C01D4B41092CC
:1006B000CD011092CE011092CF011092D0010E9474
:1006C0002E039C014427552760E074E284EF90E0FC
:1006D0000E94C719293B8DE8380786E0480780E06B
:1006E000580798F481E1E81687E2F80670F4B7013C
:1006F000882799270E94721928EE33E040E050E0E5
:100700000E94A51979018A0110C000271127CA018A
:10071000B90128EE33E040E050E00E94A519C8017D
:10072000B7010E9472197B018C018091CD019091DB
:10073000CE01A091CF01B091D00124B5BA2FA92F3D
:10074000982F8827332744275527822B932BA42BB8
:10075000B52BA80197012D0D311D411D511D82178B
:100760009307A407B50708F31F910F91FF90EF902F
:10077000DF9008951092DD011092DE011092DF01EA
:100780001092E0011092D9011092DA011092DB016F
:100790001092DC0108956091DD017091DE0180917D
:1007A000DF019091E00108951092D5011092D601D9
:1007B0001092D7011092D8011092D1011092D2015B
:1007C0001092D3011092D40108956091D5017091D7
:1007D000D6018091D7019091D8010895893031F4E4
:1007E0008FB582608FBD8FB58E7F0AC08A3019F4B5
:1007F0008FB5826002C08FB58D7F8FBD8FB5816050
:100800008FBD1BBC1ABC19BC18BC10927900109289
:10081000780008958FB580688FBD8FB58F7B8FBDB1
:1008200008958FB580628FBD8FB58F7E8FBD08957F
:100830008FB588608FBD8FB58B7F8FBD08958FB5C5
:100840008F778FBD8FB58F7B8FBD08958FB58F7DCF
:100850008FBD8FB58F7E8FBD08958FB5877F8FBD7C
:100860008FB58B7F8FBD0895292F33272BBD8ABD70
:100870000895292F332729BD88BD0895292F3327AF
:1008800020937900809378000895893049F480910D
:100890008B00826080938B0080918B008E7F0EC0D6
:1008A0008A3021F480918B00826003C080918B009C
:1008B0008D7F80938B0080918B00816080938B0073
:1008C000109287001092860010928500109284008A
:1008D00010928300109282000895EBE8F0E080818E
:1008E0008068808380818F7B80830895EBE8F0E0CF
:1008F00080818062808380818F7E80830895EBE891
:10090000F0E080818860808380818B7F8083089580
:10091000EBE8F0E080818F77808380818F7B80831C
:100920000895EBE8F0E080818F7D808380818F7E69
:1009300080830895EBE8F0E08081877F8083808169
:100940008B7F80830895292F3327209387008093FE
:1009500086000895292F33272093850080938400F3
:100960000895292F332720938300809382000895D0
:10097000EF92FF921F93CF93DF93182F7B018D315E
:10098000B0F08F3111F413E014C08E3111F414E083
:1009900010C08D3109F497C0853211F410E03CC0CD
:1009A000843211F411E038C0833219F48EC08330E0
:1009B00098F18091440186FD0BC00E94C902789491
:1009C0008AE00E94EE038091440180648093440198
:1009D00080914401C12FDD2799270C2E02C09595E7
:1009E00087950A94E2F780FD4AC087B3FE01ED5C6B
:1009F000FE4F9081892B87BB812F0E948B02209113
:100A0000440181E090E002C0880F991FCA95E2F787
:100A1000282B2093440133C08091440187FD0BC0F3
:100A20000E94EC0278948AE00E944504809144017F
:100A300080688093440180914401C12FDD2799276C
:100A40000C2E02C0959587950A94E2F780FD1DC093
:100A500082B1FE01ED5CFE4F9081892B82B9812F1E
:100A60000E948B022091440181E090E002C0880F37
:100A7000991FCA95E2F7282B2093440106C0153030
:100A800021F4C7010E94340422C0143021F4C701AC
:100A90000E9439041CC0133021F4C7010E943E0497
:100AA00016C0123021F4C7010E94A30410C01130F7
:100AB00021F4C7010E94AA040AC0112341F4C7010E
:100AC0000E94B10404C015E074CF12E0A5CFDF91FD
:100AD000CF911F91FF90EF9008951F920F920FB644
:100AE0000F9211242F933F934F935F936F937F93B4
:100AF0008F939F93AF93BF93EF93FF93809149019F
:100B000090914A01892B29F0E0914901F0914A0125
:100B10000995FF91EF91BF91AF919F918F917F9137
:100B20006F915F914F913F912F910F900FBE0F905A
:100B30001F9018951F920F920FB60F9211242F93AA
:100B40003F934F935F936F937F938F939F93AF9355
:100B5000BF93EF93FF938091D5019091D601A0911F
:100B6000D701B091D8010196A11DB11D8093D50187
:100B70009093D601A093D701B093D8018091D5016D
:100B80009091D601A091D701B091D8010097A1050D
:100B9000B10599F48091D1019091D201A091D30136
:100BA000B091D4010196A11DB11D8093D101909304
:100BB000D201A093D301B093D4018091CD01909143
:100BC000CE01A091CF01B091D0010196A11DB11D20
:100BD0008093CD019093CE01A093CF01B093D0012B
:100BE0008091530190915401892B29F0E091530198
:100BF000F09154010995FF91EF91BF91AF919F91B1
:100C00008F917F916F915F914F913F912F910F90B5
:100C10000FBE0F901F9018951F920F920FB60F9254
:100C200011242F933F934F935F936F937F938F93F1
:100C30009F93AF93BF93EF93FF9380915701909150
:100C40005801892B29F0E0915701F091580109953D
:100C5000FF91EF91BF91AF919F918F917F916F9194
:100C60005F914F913F912F910F900FBE0F901F906A
:100C700018951F920F920FB60F9211242F933F9346
:100C80004F935F936F937F938F939F93AF93BF9394
:100C9000EF93FF9380914B0190914C01892B29F0A8
:100CA000E0914B01F0914C010995FF91EF91BF91BB
:100CB000AF919F918F917F916F915F914F913F91F4
:100CC0002F910F900FBE0F901F9018951F920F92AB
:100CD0000FB60F9211242F933F934F935F936F930F
:100CE0007F938F939F93AF93BF93EF93FF938091E5
:100CF0004D0190914E01892B29F0E0914D01F09129
:100D00004E010995FF91EF91BF91AF919F918F9106
:100D10007F916F915F914F913F912F910F900FBEF7
:100D20000F901F9018951F920F920FB60F921124DB
:100D30002F933F934F935F936F937F938F939F93E3
:100D4000AF93BF93EF93FF9380914F019091500128
:100D5000892B29F0E0914F01F09150010995FF9105
:100D6000EF91BF91AF919F918F917F916F915F9123
:100D70004F913F912F910F900FBE0F901F9018959C
:100D80001F920F920FB60F9211242F933F934F9300
:100D90005F936F937F938F939F93AF93BF93EF93E3
:100DA000FF938091510190915201892B29F0E0919C
:100DB0005101F09152010995FF91EF91BF91AF91CF
:100DC0009F918F917F916F915F914F913F912F9163
:100DD0000F900FBE0F901F9018951F920F920FB695
:100DE0000F9211242F933F934F935F936F937F93B1
:100DF0008F939F93AF93BF93EF93FF938091550190
:100E000090915601892B29F0E0915501F0915601FE
:100E10000995FF91EF91BF91AF919F918F917F9134
:100E20006F915F914F913F912F910F900FBE0F9057
:100E30001F9018951F920F920FB60F9211242F93A7
:100E40003F934F935F936F937F938F939F93AF9352
:100E5000BF93EF93FF938091590190915A01892B91
:100E600029F0E0915901F0915A010995FF91EF9114
:100E7000BF91AF919F918F917F916F915F914F91B2
:100E80003F912F910F900FBE0F901F9018951F92BA
:100E90000F920FB60F9211242F933F934F935F93AE
:100EA0006F937F938F939F93AF93BF93EF93FF9332
:100EB00080914D0190914E01892B29F0E0914D01D7
:100EC000F0914E010995FF91EF91BF91AF919F91E4
:100ED0008F917F916F915F914F913F912F910F90E3
:100EE0000FBE0F901F9018951F920F920FB60F9282
:100EF00011242F933F934F935F936F937F938F931F
:100F00009F93AF93BF93EF93FF9380915D01909177
:100F10005E01892B29F0E0915D01F0915E01099558
:100F2000FF91EF91BF91AF919F918F917F916F91C1
:100F30005F914F913F912F910F900FBE0F901F9097
:100F400018951F920F920FB60F9211242F933F9373
:100F50004F935F936F937F938F939F93AF93BF93C1
:100F6000EF93FF9380915F0190916001892B29F0AD
:100F7000E0915F01F09160010995FF91EF91BF91C0
:100F8000AF919F918F917F916F915F914F913F9121
:100F90002F910F900FBE0F901F901895E5E4F1E090
:100FA00011821082329681E0E136F807C9F70E947B
:100FB000C9020E94D3020E94EC02789408958FB572
:100FC0008D7F8FBD8FB58E7F8FBD8FB58F778FBD96
:100FD0008FB58F7B8FBD8FB58F7D8FBD8FB58F7E8A
:100FE0008FBD8FB5877F8FBD8FB58B7F8FBD0895E8
:100FF000EBE8F0E080818D7F808380818E7F80832D
:1010000080818F77808380818F7B808380818F7DBB
:10101000808380818F7E80838081877F80838081B1
:101020008B7F808308959C01892B61F080917001F2
:10103000816080937001220F331F30936D012093E4
:101040006C010BC0809170018E7F8093700182E0F3
:1010500090E090936D0180936C018FB58F778FBD79
:101060008FB580648FBD8AB59BB520916E0130919C
:101070006F01820F931F9BBD8ABD87B7806187BFB9
:1010800008959C01892B61F080916B0181608093B0
:101090006B01220F331F30936801209367010BC04F
:1010A00080916B018E7F80936B0182E090E0909342
:1010B0006801809367018FB58F7D8FBD8FB580618B
:1010C0008FBD88B599B52091690130916A01820F71
:1010D000931F99BD88BD87B7886087BF08959C011D
:1010E000892B61F080916601816080936601220FF7
:1010F000331F30936301209362010BC0809166011E
:101100008E7F8093660182E090E0909363018093EC
:1011100062018FB5877F8FBD8FB584608FBD809151
:101120007800909179002091640130916501820FDF
:10113000931F909379008093780080917D00816067
:1011400080937D000895853021F4CB010E9413081F
:101150000895843021F4CB010E9441080895833022
:1011600019F4CB010E946F0808958091700181608D
:101170008093700110926D0110926C01089580911E
:101180006B01816080936B0110926801109267017E
:1011900008958091660181608093660110926301D9
:1011A00010926201089580916C0190916D010196F9
:1011B00096958795089580916701909168010196B1
:1011C00096958795089580916201909163010196AB
:1011D00096958795089580916C0190916D01892B6A
:1011E000C1F08AB59BB520916E0130916F01820FDD
:1011F000931F9BBD8ABD8091700180FF13C08091B9
:101200006C0190916D01019790936D0180936C0139
:1012100008958FB58F778FBD8FB58F7B8FBD87B7C3
:101220008F7E87BF08958091670190916801892B17
:10123000C1F088B599B52091690130916A01820F9A
:10124000931F99BD88BD80916B0180FF13C0809171
:1012500067019091680101979093680180936701FD
:1012600008958FB58F7D8FBD8FB58F7E8FBD87B76A
:10127000877F87BF08958091620190916301892BD8
:10128000E1F0809178009091790020916401309193
:101290006501820F931F909379008093780080916D
:1012A000660180FF15C080916201909163010197F2
:1012B000909363018093620108958FB5877F8FBDFE
:1012C0008FB58B7F8FBD80917D008E7F80937D0059
:1012D0000895EF92FF920F931F937C010E942303C6
:1012E000AA27BB2700271127EE0CFF1C001F111F88
:1012F000BC01CD01A80197010E9472199B01AC01AC
:1013000060E074E284EF90E00E94A51930936501DB
:10131000209364011F910F91FF90EF900895EF9239
:10132000FF920F931F937C010E942303AA27BB27E0
:1013300000271127EE0CFF1C001F111FBC01CD015F
:10134000A80197010E9472199B01AC0160E074E250
:1013500084EF90E00E94A51930936A0120936901FF
:101360001F910F91FF90EF900895EF92FF920F93CE
:101370001F937C010E942303AA27BB270027112764
:10138000EE0CFF1C001F111FBC01CD01A80197012D
:101390000E9472199B01AC0160E074E284EF90E05E
:1013A0000E94A51930936F0120936E011F910F9138
:1013B000FF90EF900895853021F4CB010E94B5098C
:1013C0000895843021F4CB010E948F090895833061
:1013D00019F4CB010E946909089510926D011092D1
:1013E0006C011092680110926701109263011092D3
:1013F00062018FB58F778FBD8FB58F7B8FBD8FB516
:101400008F7D8FBD8FB58F7E8FBD8FB5877F8FBD51
:101410008FB58B7F8FBD83E00E94450384E00E94DF
:10142000450385E00E94450308950E94C9020E9479
:10143000DF071092700110926B01109266011092FA
:101440006D0110926C011092680110926701109268
:1014500063011092620180E090E890936F018093A5
:101460006E0190936A018093690190936501809366
:1014700064016BEE78E083E00E940D0363E179E0A4
:1014800084E00E940D036BE379E085E00E940D0388
:1014900008958091610186FD07C00E94150A809120
:1014A00061018064809361010895CF92DF92EF9291
:1014B000FF921F93182F7B016A010E94490AB7010E
:1014C000812F0E94DB09B601812F0E94A3081F9182
:1014D000FF90EF90DF90CF90089540E050E00E94A1
:1014E000550A0895853029F480916C0190916D0121
:1014F0000DC0843029F4809167019091680106C085
:10150000833041F480916201909163010196969538
:10151000879508950895853051F480917001816018
:101520008093700110926D0110926C0108958430C7
:1015300051F480916B01816080936B01109268017E
:10154000109267010895833049F4809166018160AB
:1015500080936601109263011092620108958330B6
:1015600089F1843028F48130B9F0823000F50BC065
:101570008530E1F1853098F1863009F440C087303C
:1015800009F052C046C080916A008C7F862B809300
:101590006A0089B781603BC080916A00837F660FD3
:1015A000660F862B80936A0089B7826030C0809175
:1015B0006A008F7C6295607F862B80936A0089B772
:1015C000846025C080916A008F736295660F660FF4
:1015D000607C862B80936A0089B7886018C08AB7C0
:1015E0008C7F862B8ABF89B7806111C08AB7837FC1
:1015F000660F660F862B8ABF89B7806208C08AB7DC
:101600008F7C6295607F862B8ABF89B7806489BF93
:1016100008958AB78F736295660F660F607C862B7C
:101620008ABF89B7806889BF0895883058F4E82F49
:10163000FF27EE0FFF1FEF58FE4F71836083642F6B
:101640000E94AF0A08958830A0F429B7E82FFF2739
:1016500081E090E00E2E02C0880F991F0A94E2F7F5
:101660008095282329BFEE0FFF1FEF58FE4F1182F0
:10167000108208951F920F920FB60F9211242F938C
:101680003F934F935F936F937F938F939F93AF930A
:10169000BF93EF93FF938091710190917201892B19
:1016A00029F0E0917101F09172010995FF91EF919C
:1016B000BF91AF919F918F917F916F915F914F916A
:1016C0003F912F910F900FBE0F901F9018951F9272
:1016D0000F920FB60F9211242F933F934F935F9366
:1016E0006F937F938F939F93AF93BF93EF93FF93EA
:1016F0008091730190917401892B29F0E09173011D
:10170000F09174010995FF91EF91BF91AF919F9175
:101710008F917F916F915F914F913F912F910F909A
:101720000FBE0F901F9018951F920F920FB60F9239
:1017300011242F933F934F935F936F937F938F93D6
:101740009F93AF93BF93EF93FF9380917501909117
:101750007601892B29F0E0917501F09176010995C8
:10176000FF91EF91BF91AF919F918F917F916F9179
:101770005F914F913F912F910F900FBE0F901F904F
:1017800018951F920F920FB60F9211242F933F932B
:101790004F935F936F937F938F939F93AF93BF9379
:1017A000EF93FF938091770190917801892B29F035
:1017B000E0917701F09178010995FF91EF91BF9148
:1017C000AF919F918F917F916F915F914F913F91D9
:1017D0002F910F900FBE0F901F9018951F920F9290
:1017E0000FB60F9211242F933F934F935F936F93F4
:1017F0007F938F939F93AF93BF93EF93FF938091CA
:10180000790190917A01892B29F0E0917901F09189
:101810007A010995FF91EF91BF91AF919F918F91BF
:101820007F916F915F914F913F912F910F900FBEDC
:101830000F901F9018951F920F920FB60F921124C0
:101840002F933F934F935F936F937F938F939F93C8
:10185000AF93BF93EF93FF9380917B0190917C01B5
:10186000892B29F0E0917B01F0917C010995FF9192
:10187000EF91BF91AF919F918F917F916F915F9108
:101880004F913F912F910F900FBE0F901F90189581
:101890001F920F920FB60F9211242F933F934F93E5
:1018A0005F936F937F938F939F93AF93BF93EF93C8
:1018B000FF9380917D0190917E01892B29F0E09129
:1018C0007D01F0917E010995FF91EF91BF91AF915C
:1018D0009F918F917F916F915F914F913F912F9148
:1018E0000F900FBE0F901F9018951F920F920FB67A
:1018F0000F9211242F933F934F935F936F937F9396
:101900008F939F93AF93BF93EF93FF9380917F014A
:1019100090918001892B29F0E0917F01F091800165
:101920000995FF91EF91BF91AF919F918F917F9119
:101930006F915F914F913F912F910F900FBE0F903C
:101940001F901895EF92FF920F931F937B018C01CC
:1019500020E030E040E050E00E949F18882329F406
:1019600060E070E080E090E014C00E944017AA2779
:1019700097FDA095BA2FBC01CD010E94951820E0DB
:101980003EEF4FEF56E40E944D18A80197010E94C8
:101990000F191F910F91FF90EF900895AF92BF9292
:1019A000CF92DF92EF92FF920F931F937B018C01F6
:1019B00059016A010E94A21887FF10C0A80197016F
:1019C000C601B5010E940A180E94A20C9B01AC013D
:1019D000C801B7010E940B187B018C01C801B70137
:1019E0001F910F91FF90EF90DF90CF90BF90AF903D
:1019F0000895009711F00E9445170895FC0177FDA6
:101A00000CC0828193816817790738F40190F081C6
:101A1000E02DE60FF71F808101C080E0992787FD48
:101A200090950895FC01828193816817790730F4BD
:101A30000190F081E02DE60FF71F40830895FC012F
:101A4000808191810895FC01808191810895DC015C
:101A500020E030E008C0ED91FC911197E20FF31FF8
:101A600010822F5F3F4FFD01848195812817390730
:101A700090F30895EF92FF920F931F93CF93DF930C
:101A80007C01C0E0D0E00FC0F701008111810C0F94
:101A90001D1FF8018081992787FD90950E94EE19FE
:101AA000F80180832196F70182819381C817D907B5
:101AB00058F3DF91CF911F910F91FF90EF90089510
:101AC000EF92FF920F931F93CF93DF937C01C0E0BF
:101AD000D0E00FC0F701008111810C0F1D1FF8012C
:101AE0008081992787FD90950E94E819F8018083ED
:101AF0002196F70182819381C817D90758F3DF91A6
:101B0000CF911F910F91FF90EF9008950F931F9326
:101B1000FC01062F142F0190F081E02D01C01083ED
:101B2000602F772767FD7095CF010E946D17FC012C
:101B3000892BA9F71F910F910895CF93DF93FC0193
:101B4000828193814817590760F4C081D18177273A
:101B500067FD7095CE01840F951F0E946D17009749
:101B600019F48FEF9FEF02C08C1B9D0BDF91CF917B
:101B7000089540E050E00E949D0D0895CF93DF93BB
:101B8000DC01FB01EC012A813B81828193812817D2
:101B9000390718F4C0E0D0E010C0C0E0D0E06081A8
:101BA0007181281B390B8D919C91820F931F0E948C
:101BB0007917892B11F4C1E0D0E0CE01DF91CF91EC
:101BC00008951F93FC0110E0808191810E94791794
:101BD000892B09F411E0812F99271F9108950F9304
:101BE0001F93CF93DF938C01DC01CD91DC91DE015B
:101BF00001C011968C918930E1F38D30D1F38A3098
:101C0000C1F38032B1F38131A1F3FE0101900020D4
:101C1000E9F73197EC1BFD0BAF01BD01CE010E942E
:101C20005017E801E881F981DF010D900020E9F704
:101C3000AE1BBF0B129702C010821197E801E8811A
:101C4000F981EA0FFB1F80818930B1F38D30A1F358
:101C50008A3091F3803281F3813171F3DF91CF913A
:101C60001F910F910895EF92FF920F931F938C0194
:101C70007B01CB0101960E94F315F80191838083CB
:101C8000F582E48213821282C8010E94270D1F91FF
:101C90000F91FF90EF900895EF92FF920F931F9393
:101CA0008C017B01CB0101960E94F315F801918311
:101CB0008083F582E48213821282C8010E94270D7C
:101CC0001F910F91FF90EF900895AF92BF92CF9226
:101CD000DF92EF92FF920F931F937B018C015A01C9
:101CE00081E290E00E94F3156C019501AC01C801FE
:101CF000B7010E94BD17C6011F910F91FF90EF9091
:101D0000DF90CF90BF90AF900895AB01AA2797FDC9
:101D1000A095BA2FBC01CD010E94650E0895CF9306
:101D2000DF93DC01FB019A0142815381EC018A813E
:101D30009B81841B950B8217930718F4C0E0D0E0B9
:101D40000EC0C0E0D0E0608171818D919C91820FC6
:101D5000931F0E948317892B11F4C1E0D0E0CE01BC
:101D6000DF91CF910895CF93DF93DC01FB01EC016C
:101D70002A813B81828193812817390718F480E0FA
:101D800090E006C040E050E0CD010E948F0E992700
:101D9000DF91CF910895CF93DF93FC01DB01828126
:101DA00093814817590758F4C081D1816D917C9176
:101DB000CE01840F951F0E94A017009719F48FEF92
:101DC0009FEF02C08C1B9D0BDF91CF91089540E0E7
:101DD00050E00E94CB0E0895FC01808191810E9409
:101DE000A017009711F081E090E008950F931F93E2
:101DF000CF93DF93EC014A815B814F5F5F4F888116
:101E000099810E949117E881F9818A819B81E80F6D
:101E1000F91F1082DF91CF911F910F910895EF92DA
:101E2000FF920F931F938C017B01FB0182819381B1
:101E3000F801958384839383828301960E94F3152E
:101E4000F80191838083C8010E94270DF70160810A
:101E50007181C8010E94F60E1F910F91FF90EF90C3
:101E60000895EF92FF920F931F938C017B01FB016A
:101E700082819381F8019583848393838283019681
:101E80000E94F315F80191838083C8010E94270DF9
:101E9000F70160817181C8010E94F60E1F910F91B8
:101EA000FF90EF900895EF92FF920F931F93CF93BF
:101EB000DF938C017B01672B21F489E3E82E81E01D
:101EC000F82EF70101900020E9F73197EE19FF098C
:101ED000E801FB83EA83FD83EC83CF0101960E9436
:101EE000F31599838883C8010E94270DB701C801A3
:101EF0000E94F60EDF91CF911F910F91FF90EF900E
:101F00000895CF92DF92EF92FF921F93CF93DF93CA
:101F10006C017B01E9012417350714F4EA01A901DA
:101F2000F701828193818C179D0720F481E090E076
:101F30000E94011AD701ED91FC911197EC0FFD1F42
:101F4000108110826D917C91640F751FC6010E94F3
:101F5000530FD701ED91FC91EC0FFD1F1083C601CB
:101F6000DF91CF911F91FF90EF90DF90CF90089578
:101F70000F931F938C01FB01228133810E94810FFB
:101F8000C8011F910F910895EF92FF920F931F9335
:101F9000CF93DF93CDB7DEB726970FB6F894DEBFA9
:101FA0000FBECDBF7C01FB01608171818E010F5F8F
:101FB0001F4FC8010E94530FB801C7010E94C40FF0
:101FC000992726960FB6F894DEBF0FBECDBFDF91DE
:101FD000CF911F910F91FF90EF900895EF92FF9294
:101FE0000F931F93CF93DF938C017B01672B21F419
:101FF00099E3E92E91E0F92EF70101900020E9F72D
:102000003197EE19FF09E801FB83EA83FD83EC8336
:10201000CF0101960E94F31599838883C8010E941D
:10202000270DB701C8010E94F60EDF91CF911F91D5
:102030000F91FF90EF900895FF920F931F93CF930E
:10204000DF93EC01F62E2A813B818C819D8128173C
:102050003907A1F408811981C9010196880F991FD8
:102060009D838C8301960E94F31599838883B80120
:10207000CE010E94F60EC8010E949616EA81FB81ED
:10208000A881B981AE0FBF1FFC923196FB83EA8312
:1020900088819981E80FF91F1082CE01DF91CF91DD
:1020A0001F910F91FF9008950E941C1008950F93A7
:1020B0001F93CF93DF93EC018B01672B11F409E39E
:1020C00011E0F80101900020E9F73197E01BF10BD6
:1020D000FB83EA838C819D818E179F0768F4FD83C3
:1020E000EC83888199810E9496168A819B81019652
:1020F0000E94F31599838883CE010E94270DB801B1
:10210000CE010E94F60EDF91CF911F910F9108959D
:102110000F931F93CF93DF93EC018B0186179707E3
:1021200029F1FB01228133818C819D8182179307E4
:1021300070F4888199810E949616F80182819381BA
:102140009D838C8301960E94F31599838883F801FF
:10215000828193819B838A83CE010E94270DF8019F
:1021600060817181CE010E94F60E8E01C801DF915F
:10217000CF911F910F910895EF92FF920F931F93AC
:10218000CF93DF93CDB7DEB726970FB6F894DEBFB7
:102190000FBECDBF7C0160E170E08E010F5F1F4F6D
:1021A000C8010E94330EB801C7010E94881026960C
:1021B0000FB6F894DEBF0FBECDBFDF91CF911F9158
:1021C0000F91FF90EF900895EF92FF920F931F935E
:1021D000CF93DF93CDB7DEB726970FB6F894DEBF67
:1021E0000FBECDBF7C0160E170E08E010F5F1F4F1D
:1021F000C8010E94330EB801C7010E9488102696BC
:102200000FB6F894DEBF0FBECDBFDF91CF911F9107
:102210000F91FF90EF900895EF92FF920F931F930D
:10222000CF93DF93EC017B012A813B81FB0182810B
:102230009381280F391F3B832A838C819D818217CC
:10224000930788F4088119813D832C83C901019685
:102250000E94F31599838883B801CE010E94F60E7F
:10226000C8010E949616F701608171818881998169
:102270000E946217E881F9818A819B81E80FF91F2A
:102280001082CE01DF91CF911F910F91FF90EF90BF
:1022900008950E940C110895EF92FF920F931F93DF
:1022A000CF93DF93EC017B01672B21F439E3E32E1D
:1022B00031E0F32E2A813B81F70101900020E9F7FC
:1022C0003197EE19FF092E0F3F1F3B832A838C8124
:1022D0009D818217930788F4088119813D832C839F
:1022E000C90101960E94F31599838883B801CE0134
:1022F0000E94F60EC8010E949616B7018881998146
:102300000E946217E881F9818A819B81E80FF91F99
:102310001082CE01DF91CF911F910F91FF90EF902E
:102320000895EF92FF920F931F937C01CB01BA01A6
:10233000A9010E94650E8C01BC01C7010E944C11CD
:10234000C8010E949616C7011F910F91FF90EF9050
:1023500008950F931F938C012AE030E00E949111A1
:10236000C8011F910F9108950F931F938C01AB012A
:10237000662757FD6095762F2AE030E00E94911184
:10238000C8011F910F9108950F931F938C019A011B
:10239000882777FD8095982FAB01BC01C8010E946A
:1023A0009111C8011F910F9108950F931F938C01F4
:1023B0002AE030E00E949111C8011F910F91089509
:1023C0000F931F938C01AB01662757FD6095762F05
:1023D0002AE030E00E949111C8011F910F910895E9
:1023E0000E944C110895FC01662311F41082089597
:1023F00081E080830895FC01662311F41082089522
:1024000081E080830895CF93DF93CDB7DEB7219726
:102410000FB6F894DEBF0FBECDBFFC01698341E06B
:10242000BE016F5F7F4F80810E940B1521960FB612
:10243000F894DEBF0FBECDBFDF91CF910895CF934B
:10244000DF93CDB7DEB721970FB6F894DEBF0FBE8E
:10245000CDBFFC01698341E0BE016F5F7F4F80818A
:102460000E940B1521960FB6F894DEBF0FBECDBFAC
:10247000DF91CF9108952F923F924F925F926F928A
:102480007F928F929F92AF92BF92CF92DF92EF9204
:10249000FF920F931F93CF93DF93CDB7DEB7A09733
:1024A0000FB6F894DEBF0FBECDBF1C016A017B01E1
:1024B000411551056105710521F460E30E941F1269
:1024C0003EC066247724822E9924AA24BB242E01A0
:1024D0000894411C511C8201060D171DC701B6014D
:1024E000A50194010E94A519F80160830894611C5C
:1024F000711CC701B601A50194010E94A5196901CB
:102500007A01211531054105510529F77301089418
:10251000E108F1086201CE0CDF1CF60160816A302F
:1025200010F4605D01C0695CC1010E941F12089433
:10253000E108F1080894C108D108F7FEEECFA09693
:102540000FB6F894DEBF0FBECDBFDF91CF911F91C4
:102550000F91FF90EF90DF90CF90BF90AF909F9042
:102560008F907F906F905F904F903F902F90089545
:102570000F931F938C016DE00E941F126AE0C80147
:102580000E941F121F910F9108950F931F938C01AA
:102590000E940312C8010E94B8121F910F91089562
:1025A0000F931F938C010E941F12C8010E94B81242
:1025B0001F910F910895EF92FF920F931F93CF9366
:1025C000DF93EC017A018B0177FF0BC06DE20E9473
:1025D0001F1210950095F094E094E11CF11C011D70
:1025E000111D2AE0B801A701CE010E943B12DF9124
:1025F000CF911F910F91FF90EF9008950F931F932C
:102600008C010E94DB12C8010E94B8121F910F9129
:102610000895AB01662757FD6095762F0E94FE1244
:1026200008952115310521F4642F0E941F12089589
:102630002A30310519F40E94DB1208950E943B12E2
:1026400008950F931F938C010E941113C8010E94DB
:10265000B8121F910F910895AB01662757FD609541
:10266000762F0E94DB120895CF92DF92EF92FF92B5
:102670000F931F93CF93DF936C018B01EB010990B4
:102680000020E9F72197C61BD70BEE24FF240BC0CF
:10269000B8016E0D7F1D41E0F60180810E940B158F
:1026A0000894E11CF11CEC16FD0694F3DF91CF9128
:1026B0001F910F91FF90EF90DF90CF9008950F93AF
:1026C0001F938C010E943413C8010E94B8121F91FD
:1026D0000F9108950F931F938C01CB010E94230D3E
:1026E000BC01C8010E9434131F910F9108950F93EC
:1026F0001F938C010E946A13C8010E94B8121F9197
:102700000F910895FC0180810E94AA140895FC0194
:1027100080810E94411490E00895FC0180810E9414
:1027200058150895019741F46F5F7F4F29F4109277
:10273000810181E08093820108956FEF7FEF81E056
:1027400090E00E9492130895FC01578346831186FE
:1027500010867183608373836283758364830895B5
:10276000CF93DF93DC01EC01288539858E819F8131
:1027700028173907B8F4ED91FC91119761931196E0
:10278000FC93EE93888599850196998788872C819B
:102790003D818E819F81820F931FE817F90710F00A
:1027A0002D933C93DF91CF910895CF93DF93DC017C
:1027B000EC0188859985009719F48FEF9FEF18C079
:1027C000ED01EA81FB814191FB83EA8301979987BF
:1027D00088872C813D818E819F81820F931FE8170E
:1027E000F90710F03B832A83842F992787FD909562
:1027F000DF91CF910895FC01808590E00895FC0160
:1028000080859185892B19F480E090E008950280FD
:10281000F381E02D808190E008950F931F93CF9373
:10282000DF93DC01EC01488559854115510511F113
:10283000EA81FB810D911C91119770E018C0808195
:10284000861719F4862F90E017C07F5F872F90E0DE
:102850008417950778F43196ED012C813D818E81A6
:102860009F81820F931F8E179F0708F4F901E017CD
:10287000F10729F780E090E0DF91CF911F910F9150
:102880000895882331F485EF91E00E94FB1390E0D6
:10289000089581EE91E00E94FB1390E008951F924D
:1028A0000F920FB60F9211242F933F934F935F9384
:1028B0006F937F938F939F93AF93BF93EF93FF9308
:1028C0008FEF91E00E94FB13882331F08FEF91E0AE
:1028D0000E94D51380939C00FF91EF91BF91AF911F
:1028E0009F918F917F916F915F914F913F912F9128
:1028F0000F900FBE0F901F9018951F920F920FB65A
:102900000F9211242F933F934F935F936F937F9375
:102910008F939F93AF93BF93EF93FF938BEE91E0D1
:102920000E94FB13882329F08BEE91E00E94D513BF
:102930008CB9FF91EF91BF91AF919F918F917F9152
:102940006F915F914F913F912F910F900FBE0F901C
:102950001F901895882329F485EF91E00E94D513E4
:10296000089581EE91E00E94D51308951F920F9271
:102970000FB60F9211242F933F934F935F936F9352
:102980007F938F939F93AF93BF93EF93FF93609148
:102990009C0080919B0084FD04C081EE91E00E9428
:1029A000B013FF91EF91BF91AF919F918F917F9164
:1029B0006F915F914F913F912F910F900FBE0F90AC
:1029C0001F9018951F920F920FB60F9211242F93FC
:1029D0003F934F935F936F937F938F939F93AF93A7
:1029E000BF93EF93FF936CB15C9904C085EF91E0C6
:1029F0000E94B013FF91EF91BF91AF919F918F9182
:102A00007F916F915F914F913F912F910F900FBEEA
:102A10000F901F901895CF92DF92FF920F931F9304
:102A2000CF93DF93042F4423D9F1FFB6F894882382
:102A3000B1F4EB0110E09BEEC92E91E0D92E699123
:102A4000C6010E94B0131F5F1017C9F75E9A5D9B05
:102A5000FECF8BEE91E00E94D5138CB91CC0EB0128
:102A600010E08FEFC82E81E0D82E6991C6010E9438
:102A7000B0131F5F1017C9F780919B00806480938B
:102A80009B0080919B0085FFFCCF8FEF91E00E941F
:102A9000D51380939C008FB790E8F922F82AFFBEE7
:102AA000DF91CF911F910F91FF90DF90CF9008950C
:102AB000DF92EF92FF920F931F93D82E7A018B0132
:102AC000F4E0EE0CFF1C001F111FFA95D1F760E037
:102AD00074E284EF90E0A80197010E94A519A80173
:102AE0009701569547953795279562177307840781
:102AF000950748F060E074E284EF90E0A801970148
:102B00000E94A5190AC060E074E284EF90E0A80179
:102B100097010E94A51921503040832F9927DD206D
:102B2000A1F48093900029B988ED8AB940E250E081
:102B300063E871E085EF91E00E94A41340E250E069
:102B400063EA71E08BEE91E029C0809398002093B6
:102B5000990088ED80939A0080E290E00E94F3153E
:102B600090930C0280930B0280E290E00E94F31598
:102B700090930A028093090260910B0270910C02FB
:102B800042E050E081EE91E00E94A41360910902BE
:102B900070910A0242E050E08FEF91E00E94A4138E
:102BA0001F910F91FF90EF90DF90089561E0809169
:102BB000C3010E94460168EE73E080E090E00E944D
:102BC000DB0060E08091C3010E94460168EE73E083
:102BD00080E090E00E94DB00089561E08091C301F5
:102BE0000E9400010895CF93DF93AC01029710F487
:102BF00042E050E0A0910F02B0911002FD01C0E050
:102C0000D0E020E030E020C08081918184179507DA
:102C100069F482819381209719F09B838A8304C091
:102C20009093100280930F02CF0132C048175907CA
:102C300038F42115310519F08217930708F49C0127
:102C4000EF010280F381E02D3097F1F62115310577
:102C500089F1C901841B950B049708F4A901E0E0F0
:102C6000F0E026C08D919C91119782179307E9F4AB
:102C70004817590779F4ED018A819B81309719F043
:102C80009383828304C09093100280930F02CD013E
:102C9000029649C0841B950BFD01E80FF91F419373
:102CA000519302978D939C933AC0FD01A281B38109
:102CB0001097C1F680910D0290910E02892B41F47C
:102CC00080913C0190913D0190930E0280930D0202
:102CD00020913E0130913F012115310541F42DB77E
:102CE0003EB780913A0190913B01281B390BE0914E
:102CF0000D02F0910E022E1B3F0B2417350788F0B2
:102D0000CA0102962817390760F0CF01840F951F7A
:102D1000029690930E0280930D0241935193CF013E
:102D200002C080E090E0DF91CF910895CF93DF93D0
:102D3000009709F44EC0EC0122971B821A82A091E1
:102D40000F02B0911002109711F140E050E001C065
:102D5000DC01AC17BD0700F1BB83AA83FE01219102
:102D60003191E20FF31FEA17FB0771F42E5F3F4F1B
:102D70008D919C911197820F931F99838883FD01F8
:102D8000828193819B838A834115510559F4D093A5
:102D90001002C0930F021DC0FD0182819381AD011D
:102DA0000097B1F6FA01D383C28321913191E20FEA
:102DB000F31FEC17FD0769F42E5F3F4F888199815F
:102DC000820F931FFA01918380838A819B81938371
:102DD0008283DF91CF910895AF92BF92CF92DF921D
:102DE000EF92FF920F931F93CF93DF93EC01E88054
:102DF000F9800A811B81C801B7012DE133EF41E061
:102E000050E00E94A51927EA31E440E050E00E941A
:102E100072195B016C01C801B7012DE133EF41E08C
:102E200050E00E94A519CA01B90124E13BE040E04D
:102E300050E00E947219A61AB70AC80AD90A1A14D1
:102E40001B041C041D0444F08FEF9FEFAFEFBFE79E
:102E5000A80EB91ECA1EDB1EA882B982CA82DB82F6
:102E6000C5019F77DF91CF911F910F91FF90EF9058
:102E7000DF90CF90BF90AF9008950E94EC16089518
:102E800080E491E00E94EC160895AA27BB27809366
:102E9000400190934101A0934201B09343010895F2
:102EA0006817790768F4FB01DC01E40FF51FA40F34
:102EB000B51F02C002900E9241505040D8F70895BD
:102EC0000C94F117FB01DC010D900020E9F711973C
:102ED00001900D920020E1F70895FC010190061683
:102EE00029F00020D9F78827992708953197CF0135
:102EF0000895FB01DC018D910190801911F40020EF
:102F0000D1F7990B0895FB01DC014150504030F09E
:102F10008D910190801919F40020B9F7881B990B45
:102F20000895FB01DC014150504048F001900D92A2
:102F30000020C9F701C01D9241505040E0F70895AC
:102F4000DC01FB014191442309F40895FB01419107
:102F50002D91222369F02417CD01D1F7419144230B
:102F600051F02C91222321F0241781F71196F6CFEE
:102F700088279927089501970895FA01CF93FF9321
:102F8000EF93223044F1253234F5C22FE894CA3051
:102F900049F497FB3EF490958095709561957F4F2D
:102FA0008F4F9F4F2C2F332744275527FF93EF93A5
:102FB0000E94A519EF91FF91605D6A330CF0695D85
:102FC0006193B901CA01605070408040904051F750
:102FD00016F4CDE2C19310828F919F91CF910C9402
:102FE000FA17FB01DC0102C001900D9241505040E4
:102FF000D8F70895DC01FC0101900020E9F7329731
:10300000AE17BF0730F47C916081708331976D9368
:10301000F7CF08955058192ED4D001D0B7C0BA17A1
:103020006207730784079507B1F188F40EF41094D2
:103030000B2EBA2FA02D062E622F202D072E732FB8
:10304000302D082E842F402D092E952F502DFF272F
:103050005523B9F0591B49F0573E98F046953795DE
:103060002795A795F0405395C9F776F0BA0F621FE0
:10307000731F841F30F4879577956795B795F04057
:10308000939517FA0F2E0895BF1BBB27BA0B620B3F
:10309000730B840BF6CFDEF6C0C093D001D076C0A0
:1030A000552359F0992369F09F575F57951B33F4C7
:1030B00042F4903811F4915805C080C091589F3F58
:1030C00009F4ABC0BB27112462177307840730F4DF
:1030D000660F771F881FBB1F915098F311D00F9276
:1030E0000FD00F920DD0A0E82617370748071B0610
:1030F00009F0A048BA2F602D7F918F910024089588
:10310000A0E80024621773078407B10528F0621B4A
:10311000730B840BB1090A2A660F771F881FBB1F28
:10312000A69581F70895E89403C097FB0EF4D2D0DA
:10313000B62F672F782F892F9EE9002427C00ED045
:103140005EF004C00BD026F001C008D019F020F4C6
:103150008FEF089580E0089581E0089597FB092E90
:10316000052600F8689430D0E89407FC07C0621781
:1031700073078407950721F008F400940794989446
:1031800008959A95BB0F661F771F881F11249923F6
:10319000A1F08823B2F79F3F59F0BB0F48F421F408
:1031A000002011F460FF04C06F5F7F4F8F4F9F4F6F
:1031B000881F9795879597F908952CC09FEF80EC0D
:1031C0000895052E092607FA440F551F5F3F79F031
:1031D000AA27A51708F051E04795880F991F9F3F30
:1031E00031F0BB27B91708F091E0879508959F91BA
:1031F0009F911124E3CF97FB880F991F9F3F31F0D8
:10320000BB27B91708F091E0879508959F919F918A
:103210001124D4CF66277727882799270895D1DFEF
:1032200001D0B4CF992339F0552329F09F575F5728
:10323000950F13F49AF1F1CF91589F3FE1F3629FFC
:10324000A12D0F92BB27639FA00DB11DEE27729F8A
:10325000A00DB11DEE1FAF93AA27649FB00DE11D15
:10326000739FB00DE11DAA1F6627829FB00DE11D5F
:10327000A61F5527749FE00DA11D551F839FE00DCC
:10328000A11D561F849FA00D511D852F7A2F6E2FD3
:103290001F900F9088231AF4939539F48FCF000C68
:1032A000111CBB1F661F771F881F0128089597FBFD
:1032B00094DF9F3738F0FEE9F91B982F872F762F80
:1032C0006B2F05C0A7CF9695879577956795F15099
:1032D000D0F73EF490958095709561957F4F8F4F14
:1032E0009F4F0895629FD001739FF001829FE00D70
:1032F000F11D649FE00DF11D929FF00D839FF00D75
:10330000749FF00D659FF00D9927729FB00DE11D20
:10331000F91F639FB00DE11DF91FBD01CF011124FD
:103320000895AA1BBB1B51E107C0AA1FBB1FA6170C
:10333000B70710F0A61BB70B881F991F5A95A9F75E
:1033400080959095BC01CD010895A1E21A2EAA1B8B
:10335000BB1BFD010DC0AA1FBB1FEE1FFF1FA21745
:10336000B307E407F50720F0A21BB30BE40BF50B42
:10337000661F771F881F991F1A9469F760957095CB
:10338000809590959B01AC01BD01CF01089597FBFD
:10339000092E05260ED057FD04D0D7DF0AD0001C19
:1033A00038F450954095309521953F4F4F4F5F4FE2
:1033B0000895F6F790958095709561957F4F8F4FA2
:1033C0009F4F0895EE0FFF1F0590F491E02D099493
:1033D0008F930CD08F9109F0806208958F9306D05F
:1033E0008F9109F08F7D089585FD08C0806291114D
:1033F00005C08136ECF38B37DCF7089599278827D1
:103400000895FFCF010204081020408032003500EB
:103410003B003800230062006500310034003A00B0
:1034200037002200610064003000330039003600AC
:1034300021002000630001201008804020002000AF
:103440001102000001000000FFFFFFFFFFFFFFFF70
:10345000FFFFFFFFFFFFFFFFFFFFFFFFFFFFFFFF7C
:10346000FFFFFFFFFFFFFFFFFFFFFFFFFFFFFFFF6C
:10347000FFFFFFFFFFFFFFFFFFFFFFFFFFFFFFFF5C
:10348000FFFFFFFFFFFFFFFFFFFFFFFFFFFFFFFF4C
:020000021000EC
:10F800000C9446FC0C9463FC0C9463FC0C9463FC19
:10F810000C9463FC0C9463FC0C9463FC0C9463FCEC
:10F820000C9463FC0C9463FC0C9463FC0C9463FCDC
:10F830000C9463FC0C9463FC0C9463FC0C9463FCCC
:10F840000C9463FC0C9463FC0C9463FC0C9463FCBC
:10F850000C9463FC0C9463FC0C9463FC0C9463FCAC
:10F860000C9463FC0C9463FC0C9463FC0C9463FC9C
:10F870000C9463FC0C9463FC0C9463FC0C9463FC8C
:10F880000C9463FC0C9463FC0C9463FC11241FBE69
:10F89000CFEFD0E1DEBFCDBF11E0A0E0B1E0ECEEF4
:10F8A000FFEF01E00BBF02C007900D92A030B1073F
:10F8B000D9F712E0A0E0B1E001C01D92A434B10775
:10F8C000E1F70C94AEFC0C9400FC0F93EF93FF93C4
:10F8D00040D0FC01062F36D0FF91EF910F91089593
:10F8E0000F930F921F92EF93FF9333D0FC010B0104
:10F8F00001E028D0FF91EF911F900F900F91089594
:10F900000F930F92EF93FF9324D0FC0160FD60935F
:10F910006800D895802DE395D895902DFF91EF91B3
:10F920000F900F9108950F930F9213D0082E09E0B6
:10F9300009D00F900F9108950F930BD001E102D0E1
:10F940000F910895E199FECF00936800E895FFFFBD
:10F9500000000091680000FDFCCF0895CFEFD0E1DA
:10F96000DEBFCDBFC6E4F8948EEF9FE00E94EDFFAE
:10F97000843B61F48FEF9FE00E94EDFF833C31F404
:10F980008DEF9FE00E94EDFF80936F000E94D8FFF3
:10F990000E94E5FF84E690E00E9482FF0E94E8FF5B
:10F9A000882311F4C150B1F7CC2319F00E94E4FC74
:10F9B00002C00E94DFFC80E090E00C94F5FF0E9402
:10F9C000DDFF0C940000089569E081E090E00E9462
:10F9D00080FC84FF03C08F7E0E9493FC0E94E8FF9E
:10F9E0008823E1F30E94E5FF992782359105DCF435
:10F9F000803591050CF054C08134910509F45AC04A
:10FA0000823491053CF48033910509F449C0C197D3
:10FA100059F136C18234910509F45FC085349105EE
:10FA200009F45EC02DC18635910509F4EDC0873516
:10FA300091054CF48235910509F461C08535910535
:10FA400009F465C01DC18437910509F4A0C085374C
:10FA500091052CF48436910509F472C011C18537E3
:10FA6000910509F4C1C00CC10E9444FE882309F429
:10FA7000B5CF84E10E94E0FF81E40E94E0FF86E5CB
:10FA80000E94E0FF82E50E94E0FF80E20E94E0FF2A
:10FA900083E50E94E0FF84E50E94E0FF8BE406C05E
:10FAA0000E9444FE882309F499CF84E10E94E0FF7C
:10FAB00080E1E7C061E070E080E091E00E9496FFA5
:10FAC0000E9444FE882309F489CF84E10E94E0FF6C
:10FAD000809100010E9456FEE9CF64E170E00AC007
:10FAE00061E070E080E091E00E9496FF809100016B
:10FAF0009927BC0180E091E00E9496FFD1CF0E943F
:10FB000044FE882309F46ACF0E94BDFECECF62E096
:10FB100070E080E091E00E9496FF0E9444FE8823FE
:10FB200009F45CCF20910001809101019927982F61
:10FB30008827820F911D9093430280934202B5CF94
:10FB400063E070E080E091E00E9496FF2091010167
:10FB5000809100019927982F8827820F911D9093FB
:10FB6000410180934001BC0182E491E00E9496FF34
:10FB70000E9444FE882309F431CF8091020186342B
:10FB800019F40E94E6FE91CF0E9473FE8ECF63E0CF
:10FB900070E080E091E00E9496FF20910101809149
:10FBA00000019927982F8827820F911D909341017A
:10FBB000809340010E9444FE882309F40FCF809176
:10FBC0000201863419F40E944BFF02C00E949AFE83
:10FBD00084E10E94E0FF609140017091410182E464
:10FBE00091E00E94B9FF64CF0E9444FE882309F48B
:10FBF000F5CE84E10E94E0FF8EE10E94E0FF87E9FC
:10FC00000E94E0FF82E052CF64E070E080E091E08B
:10FC10000E9496FF0E9444FE882309F4DFCE84E10F
:10FC20000E94E0FF90910001903541F48091010124
:10FC3000882321F469E080E090E01FC0983541F40A
:10FC400080910101883021F469E083E090E015C0E3
:10FC5000903541F480910101883021F469E082E01F
:10FC600090E00BC0983509F023CF809101018823E3
:10FC700009F01ECF69E081E090E00E9480FC16CF81
:10FC800085E10E94E0FFAACE0E94E8FF8823E1F30D
:10FC90000E94E5FF803219F481E090E0089585E14B
:10FCA0000E94E0FF80E090E00895089590E0282F02
:10FCB00033272138310589F02238310524F42038E2
:10FCC000310549F00DC02238310549F02839310598
:10FCD00039F493E005C092E003C091E001C09FE0D9
:10FCE000892F9927089540E050E06091400170917C
:10FCF000410146175707E8F4E2E4F1E0809142023F
:10FD00008EBB8091420290914302292F33272FBB53
:10FD10000196909343028093420280818DBBE29AC8
:10FD2000E19AE199FECF4F5F5F4F31964617570733
:10FD300028F3089540E050E0609140017091410146
:10FD400046175707C8F4E2E4F1E0809142028EBB07
:10FD50008091420290914302292F33272FBB0196B5
:10FD60009093430280934202E09A8DB381934F5F58
:10FD70005F4F4617570748F308950F931F93CF938C
:10FD8000DF9300E010E0E801D0934302C093420209
:10FD9000D7FF03C081E08BBF01C01BBE8091420230
:10FDA00090914302880F991F63E00E9465FC0F5FEA
:10FDB0001F4FC058DF4F82E00030180728F30E9421
:10FDC0009CFCDF91CF911F910F910895EF92FF92CC
:10FDD0000F931F93CF93DF93809142029091430240
:10FDE00097FF03C081E08BBF01C01BBE00E010E0A5
:10FDF00080914001909141010817190708F044C013
:10FE0000EE24FF24E801CE5BDE4F488189819927EB
:10FE1000382F2227240F311D8091420290914302F6
:10FE2000880F991F8E0D9F1DB9010E9470FC82E002
:10FE300090E0E80EF91EC80FD91F9FEFE916F104F4
:10FE400021F318F38091420290914302880F991F89
:10FE5000800F911F63E00E9465FC809142029091A7
:10FE60004302880F991F800F911F65E00E9465FC77
:10FE70000E949CFC00501F4F8091400190914101D5
:10FE80000817190708F4BCCFDF91CF911F910F918C
:10FE9000FF90EF9008950F931F93CF93DF9380917E
:10FEA00042029091430297FF03C081E08BBF01C0E3
:10FEB0001BBE00E010E080914001909141010817C5
:10FEC0001907D8F4C2E4D1E0809142029091430234
:10FED000880F991F800F911F60E00E9480FC88832B
:10FEE000892F992789830E5F1F4F229680914001A9
:10FEF000909141010817190738F3DF91CF911F91B5
:10FF00000F91089540E050E04817590770F420E041
:10FF100030E000002F5F3F4F67E0203D3607C8F319
:10FF20004F5F5F4F4817590790F30895EF92FF9284
:10FF30000F931F93CF93DF937B01C0E0D0E0C617F0
:10FF4000D70770F48C010E94E8FF8823E1F30E9438
:10FF5000E5FFF80181938F012196CE15DF0598F317
:10FF600081E090E0DF91CF911F910F91FF90EF9092
:10FF70000895EF92FF920F931F93CF93DF938C011D
:10FF80007B01C0E0D0E0C617D70748F4F8018191A3
:10FF90008F010E94E0FF2196CE15DF05B8F381E0C6
:10FFA00090E0DF91CF911F910F91FF90EF90089516
:10FFB00088E089B9549A539A0895549853980895AB
:10FFC0008CB95E9BFECF5E9A08958CB199270895F7
:10FFD0008BB19927807890700895E199FECF9FBBEF
:10FFE0008EBBE09A99278DB30895FFCFFFFFFFFFE7
:10FFF000FFFFFFFFFFFFFFFFFFFFFFFFFFFFFFFF11
:00000001FF
